:100000000C9468000C9490000C9490000C94900058
:100010000C9490000C9490000C9490000C94900020
:100020000C9490000C9490000C9490000C94900010
:100030000C9490000C9490000C9490000C94900000
:100040000C9477110C9490000C946C140C949E14E6
:100050000C9490000C9490000C9490000C949000E0
:100060000C9490000C949000000000080002010025
:100070000003040700000000000000000000000171
:10008000020408102040800102040810200102042C
:100090000810204080400404040404040404020204
:1000A000020202020303030303030202030000002F
:1000B0000023002600290000000000250028002B56
:1000C0000000000000240027002A00001F11CE14A9
:1000D00011241FBECFEFD8E0DEBFCDBF12E0A0E0FD
:1000E000B1E0E4E2FCE202C005900D92A431B10758
:1000F000D9F724E0A4E1B2E001C01D92AD33B2070C
:10010000E1F710E0C8E6D0E004C02197FE010E94AC
:10011000FB15C636D107C9F70E9468150C94101656
:100120000C940000CF92DF92EF92FF920F931F93F7
:10013000E82FF92F05C0015011092109310961F19A
:10014000908196239417B9F305C001501109210934
:10015000310911F1908196239413F7CFC12CD12C42
:10016000E12CF12C0AC08FEFC81AD80AE80AF80A65
:100170000C151D052E053F0579F080818623841717
:1001800091F36C2D7D2D8E2D9F2D1F910F91FF9042
:10019000EF90DF90CF90089560E070E080E090E015
:1001A0001F910F91FF90EF90DF90CF900895DC01A9
:1001B000ED91FC910190F081E02D09940F931F9334
:1001C000CF93DF930CEC12E0C0E0D0E06C2F6170B5
:1001D00084E00E949512BE0175956795617083E079
:1001E0000E949512BE01759567957595679582E099
:1001F0000E94951283E10E941312F801819391935A
:100200008F012196C830D10509F7DF91CF911F9159
:100210000F910895EF92FF920F931F93CF93DF9367
:1002200090912801E0912F018091B2022091B302B8
:10023000992361F1F0E0EF01CB5CDD4F90912B0150
:100240003CE0939F800D112488834DE0249F900112
:100250001124D901AD5CBE4F1C96EC90F12C00E04E
:1002600010E0C801B7010E948715D901A80FB91F76
:10027000AD5CBE4F9C918881890F8A930F5F1F4FA1
:10028000CF01801B910B019661F72AC090912D013F
:10029000BCE09B9F800D112480933502F0E005E3C4
:1002A00012E0C0E0D0E04DE0249F90011124D9017C
:1002B000A15CBE4FEC90F12CD8014D918D01CE0187
:1002C000B7010E948715D901A80FB91FAD5CBE4FB9
:1002D0008C91480FD8014C932196EC17FD0764F7D9
:1002E000DF91CF911F910F91FF90EF9008951F9391
:1002F000CF93DF931F92CDB7DEB7282F862F142F11
:1003000060E029830E94951260E08EE00E949512C1
:10031000298141E06FE089E00E94F71261E08EE000
:100320000E94951261E0812F0F90DF91CF911F9174
:100330000C949512CF93DF93EC011C161D0664F507
:10034000E091CB02F0E0E153FE4F42E160E18081B9
:100350000E94770184EF91E00E94CD11E091CA02E2
:10036000F0E0E153FE4F41E162E180810E947701BC
:1003700084EF91E00E94CD11E091C902F0E0E153D9
:10038000FE4F40E161E180810E94770184EF91E0BE
:100390000E94CD112197D1CFDF91CF9108959C017B
:1003A0008A3091055CF0EAE0F0E0BF010E94871519
:1003B000CB01BF010E948715982F01C096E1909351
:1003C000CA02C9016AE070E00E9487158093C902E1
:1003D00008959C01843691055CF064E670E00E940B
:1003E0008715CB016AE070E00E948715982F01C045
:1003F00096E19093CB02C9010C94CF010F931F9308
:10040000CF93C82F0E94C1116093C5027093C6029A
:100410008093C7029093C80200913001109131017E
:10042000012E000C220B330B060F171F281F391F3C
:100430000093C1021093C2022093C3023093C402FE
:10044000DC01CB01805A9541AF4FBF4F8093BD0275
:100450009093BE02A093BF02B093C002C093BC02AF
:10046000CF911F910F9108959B012E5F3F4F281749
:1004700039075CF0625071098617970744F4892F99
:100480008095881F8827881F089581E0089580E05F
:1004900008958091B30290E001960E94CF0180916F
:1004A000B202865F8093CB020895AF92BF92CF9243
:1004B000DF92EF92FF920F931F93CF93DF93EC01A4
:1004C000CC0FDD1FFE01E453FD4F608171818091EF
:1004D0001401909115016817790709F45EC0072E81
:1004E000000C880B990B1F921F921F922CE02F93E8
:1004F000A12CB12C6501EE24EA9413E0F12E00E06A
:1005000010E020E030E0A9010E9426150F900F9026
:100510000F900F906C3018F46093B30203C08BE01F
:100520008093B302E091B3028DE0E89FF0011124C3
:10053000ED5CFE4F909129016485969F602D1124FA
:1005400060932F0170E080ED92E00E948715709318
:10055000B1026093B0020E940A01FE01E453FD4F14
:100560006081718180911401909115010E94340283
:10057000882321F08091BC02833048F0C453DD4FC2
:1005800088819981909315018093140106C082E0BF
:100590000E94FE010E944902F1CFDF91CF911F918D
:1005A0000F91FF90EF90DF90CF90BF90AF900895A4
:1005B000AF92BF92CF92DF92EF92FF920F931F9371
:1005C000CF93DF93EC01CC0FDD1FFE01E453FD4F11
:1005D00060817181809112019091130168177907F0
:1005E00009F445C0072E000C880B990B1F921F922F
:1005F0001F922CE02F93A12CB12C6501EE24EA94DC
:1006000013E0F12E00E010E020E030E0A9010E94AC
:1006100026150F900F900F900F906C3018F4609388
:10062000B20203C08BE08093B2020E940A01FE0175
:10063000E453FD4F6081718180911201909113010B
:100640000E943402882321F08091BC02833048F05C
:10065000C453DD4F888199819093130180931201D7
:1006600006C082E00E94FE010E944902F1CFDF91A4
:10067000CF911F910F91FF90EF90DF90CF90BF909F
:10068000AF9008958F929F92AF92BF92CF92DF92D8
:10069000EF92FF920F931F93CF93DF93EB014C01E7
:1006A000880C991CF401E453FD4F608171818091A5
:1006B000100190911101CC0FDD1F6817790769F4C3
:1006C000FE01E453FD4F2081318180910E01909114
:1006D0000F012817390759F502C1072E000C880BA6
:1006E000990B1F921F921F922AE02F93A12CB12CDD
:1006F0006501A394EE24EA9413E0F12E00E010E0EB
:1007000020E030E0A9010E9426150F900F900F9075
:100710000F90693071052CF470932E0160932D01B8
:1007200006C088E090E090932E0180932D01FE0199
:10073000E453FD4F6081718180910E0190910F0112
:100740006817790751F1072E000C880B990B1F923F
:100750001F921F922AE02F93A12CB12C6501A39424
:10076000EE24EA9413E0F12E00E010E020E030E007
:10077000A9010E9426150F900F900F900F906930DD
:1007800071052CF470932C0160932B0106C088E056
:1007900090E090932C0180932B0120912B013091BC
:1007A0002C0180912D0190912E01A901485F5F4F8E
:1007B000481B590B50930D0140930C0148305105D3
:1007C00041F440910A0150910B0150930D01409367
:1007D0000C0140910C0150910D014830510524F459
:1007E00041E04093280105C04830510511F01092B6
:1007F00028018217930754F0582F492F28173907DB
:1008000014F4522F432F9C01852F942F281B390B52
:100810002F5F3F4F30932A0120932901E091B302CB
:100820008DE0E89FF0011124ED5CFE4F6485629F2E
:10083000202D112420932F01622F70E080ED92E093
:100840000E9487157093B1026093B0020E940A0162
:10085000FE01E453FD4F6081718180910E01909102
:100860000F010E94340281112BC0F401E453FD4FAB
:100870006081718180911001909111010E94340278
:10088000882321F08091BC028330D0F0F401E4533E
:10089000FD4F808191819093110180931001C45389
:1008A000DD4F8881998190930F0180930E01809193
:1008B0000C0190910D0190930B0180930A010FC0E0
:1008C00082E00E94FE0180912D018093CB028091F5
:1008D0002B018093C90286E18093CA02D7CFDF91B2
:1008E000CF911F910F91FF90EF90DF90CF90BF902D
:1008F000AF909F908F90089581E08093A40280E252
:1009000093E0909331018093300108951092A402F6
:1009100080ED97E090933101809330010895AF927C
:10092000BF92CF92DF92EF92FF920F931F93CF93DC
:10093000DF93EC01CC0FDD1FFE01E453FD4F60811E
:10094000718180910801909109016817790709F474
:1009500062C0072E000C880B990B1F921F921F92EA
:1009600028E02F93A12CB12C6501A394EE24EA94E6
:1009700013E0F12E00E010E020E030E0A9010E9439
:1009800026150F900F900F900F90683018F4609319
:10099000AD0203C087E08093AD02FE01E453FD4F3A
:1009A0006081718180910801909109010E94340257
:1009B0008823B1F083E00E94FE0186E18093C902A2
:1009C0008093CA028091AD028093CB028FEF9FEF9C
:1009D0009093250180932401909327018093260111
:1009E0008091AD02863031F48091A402811102C061
:1009F0000E947C048091AD02863029F08091A4028F
:100A000081110E948604C453DD4F8881998190939F
:100A1000090180930801DF91CF911F910F91FF9001
:100A2000EF90DF90CF90BF90AF9008956F927F923C
:100A30008F929F92AF92BF92CF92DF92EF92FF92EE
:100A40000F931F93CF93DF933B014C01880C991CAC
:100A5000E401C453DD4F6881798180913302909124
:100A600034028617970771F1072E000C880B990B3B
:100A70001F921F921F922FE72F93A12CB12C65017B
:100A8000EE24EA9413E0F12E00E010E020E030E0E4
:100A9000A9010E94261570932301609322016881A9
:100AA000798180913302909134020E9434020F9038
:100AB0000F900F900F90882329F08091BC02833013
:100AC00008F45FC0E301CC0FDD1FCE0184539D4FBE
:100AD0003C01FC0160817181809131029091320270
:100AE0008617970771F1072E000C880B990B1F9240
:100AF0001F921F922FE72F93A12CB12C6501EE249A
:100B0000EA9413E0F12E00E010E020E030E0A901CB
:100B10000E9426157093210160932001F3016081EA
:100B2000718180913102909132020E9434020F90C3
:100B30000F900F900F90882321F08091BC0283309A
:100B400050F1F401E453FD4F808191819093340280
:100B500080933302C453DD4F888199819093320290
:100B600080933102DF91CF911F910F91FF90EF9011
:100B7000DF90CF90BF90AF909F908F907F906F90BD
:100B8000089582E00E94FE0180912201909123014C
:100B90000E94E90197CF82E00E94FE01809120012E
:100BA000909121010E94E901CCCF6F927F928F92A8
:100BB0009F92AF92BF92CF92DF92EF92FF920F93EC
:100BC0001F93CF93DF934C01EB01CC0FDD1FCE01C0
:100BD00084539D4F3C01FC0160817181809106012D
:100BE000909107018617970779F1072E000C880B63
:100BF000990B1F921F921F922FE72F93A12CB12CBC
:100C00006501EE24EA9413E0F12E00E010E020E00C
:100C100030E0A9010E9426157093A8026093A702F4
:100C2000F3016081718180910601909107010E941A
:100C300034020F900F900F900F90882329F080912D
:100C4000BC02833008F45EC0880C991CC401845334
:100C50009D4F3C01FC016081718180910401909164
:100C600005018617970771F1072E000C880B990B69
:100C70001F921F921F922FE72F93A12CB12C650179
:100C8000EE24EA9413E0F12E00E010E020E030E0E2
:100C9000A9010E9426157093A6026093A502F30194
:100CA0006081718180910401909105010E9434025C
:100CB0000F900F900F900F90882321F08091BC022D
:100CC000833050F1C453DD4F88819981909307019F
:100CD00080930601F401E453FD4F8081918190934C
:100CE000050180930401DF91CF911F910F91FF9037
:100CF000EF90DF90CF90BF90AF909F908F907F90BC
:100D00006F90089582E00E94FE018091A702909169
:100D1000A8020E94E90198CF82E00E94FE01809122
:100D2000A5029091A6020E94E901CCCF8091B30266
:100D300090E001960E94CF018091B202865F80937D
:100D4000CB021092BC02089586E18093CB0280937F
:100D5000CA028093C90208950F931F930E94C11184
:100D60006093C5027093C6028093C7029093C80235
:100D70000091BD021091BE022091BF023091C002CD
:100D8000061717072807390720F41F910F910C94B5
:100D9000A4060091C1021091C2022091C3023091B9
:100DA000C402061717072807390768F40E94960639
:100DB0008091A402882339F08FE28093CB02809344
:100DC000CA028093C9021F910F910895AF92BF92FA
:100DD000CF92DF92EF92FF920F931F9380911F01AA
:100DE000882309F452C061E084E00E94951261E01A
:100DF00083E00E94951261E082E00E94951283E1F7
:100E00000E941312BC019093DB028093DA0280915E
:100E10002F029091300268177907B9F1072E000C64
:100E2000880B990B1F921F921F9221E12F93A12CE7
:100E3000B12C6501A394EE24EA9413E0F12E00E0B6
:100E400010E020E030E0A9010E94261560931E0109
:100E50008091DA029091DB029093300280932F020E
:100E60002FE0629FC00111240E94E9010F900F90B2
:100E70000F900F9083E01F910F91FF90EF90DF9004
:100E8000CF90BF90AF900C94FE011F910F91FF90F7
:100E9000EF90DF90CF90BF90AF90089561157105EE
:100EA0008105910581F06F3521E07207810591057B
:100EB0006CF0683B2BE072078105910554F4462FD6
:100EC000372F282F0AC040E030E005C04EE531E062
:100ED00002C048EB3BE020E090E0642F732F822FAC
:100EE0000895CF93DF93C82FD62F60E00E9495120C
:100EF00082E090E00E94CD1161E08C2F0E9495125B
:100F00008AE090E00E94CD1160E08C2F0E94951243
:100F100020EA3FE040E050E061E08D2FDF91CF918B
:100F20000C94C5126115710581059105B1F12091EF
:100F30002E02E22FF0E0EE0FFF1FEA5DFD4F7183FE
:100F4000608381E0820F843018F480932E0202C007
:100F500010922E0260912602709127028091280241
:100F600090912902680F791F80912A0290912B029B
:100F7000680F791F80912C0290912D02680F791FC4
:100F800077FF02C06D5F7F4F759567957595679583
:100F9000072E000C880B990B089560E070E0CB01E0
:100FA00008956115710581059105B1F12091250222
:100FB000E22FF0E0EE0FFF1FE35EFD4F71836083D1
:100FC00081E0820F843018F48093250202C01092D1
:100FD000250260911D0270911E0280911F02909166
:100FE0002002680F791F8091210290912202680FE0
:100FF000791F8091230290912402680F791F77FF57
:1010000002C06D5F7F4F7595679575956795072E43
:10101000000C880B990B089560E070E0CB010895F7
:101020004F925F926F927F92AF92BF92CF92DF9278
:10103000EF92FF920F931F936091B8027091B902E3
:101040008091BA029091BB026115710581059105ED
:10105000C9F1A090A902B090AA020B2C000CCC08F8
:10106000DD082091AB023091AC022901330F6608F4
:1010700077087F926F925F924F9218EBE12E1BE000
:10108000F12E00E010E02EE531E040E050E00E945B
:10109000261560931701862F90E00E94E9010F90BA
:1010A0000F900F900F9081E01F910F91FF90EF90A4
:1010B000DF90CF90BF90AF907F906F905F904F90F8
:1010C0000C94FE011F910F91FF90EF90DF90CF9055
:1010D000BF90AF907F906F905F904F9008954F9228
:1010E0005F926F927F92AF92BF92CF92DF92EF9218
:1010F000FF920F931F93CF93DF932B013C01E0905E
:101100002F01F12C8FEFE81AF80A0F2C000C000BBE
:10111000110B6091AE027091AF026F5F7F4F072E8F
:10112000000C880B990B1F921F92DBE0DF93C8EB3A
:10113000CF932EE5A22EBB24B394C12CD12C20E05A
:1011400030E0A9010E9426152091B0023091B10231
:101150008901330F220B330BDC01CB01800F911F70
:10116000A21FB31F0F900F900F900F90841595053D
:10117000A605B7050CF449C0E0902F01F12C8FEFC4
:10118000E81AF80A0F2C000C000B110B6091AE024C
:101190007091AF02072E000C880B990B1F921F92C3
:1011A000DF93CF9320E030E0A9010E942615009143
:1011B000B0021091B102012E000C220B330BDC01A6
:1011C000CB01801B910BA20BB30B0F900F900F90D4
:1011D0000F90481659066A067B06BCF06091B4026F
:1011E0007091B5028091B6029091B702DF91CF91D4
:1011F0001F910F91FF90EF90DF90CF90BF90AF9035
:101200007F906F905F904F9008954092B4025092FB
:10121000B5026092B6027092B702E0CF68E087E054
:101220000E9471070E944E070C946F080F931F9342
:10123000CF9303E010E0C4E2C093CB02C093CA0294
:10124000C093C9028EE190E00E949A01CF5FCD3237
:1012500099F70E940E096093B4027093B5028093CF
:10126000B6029093B7020150110929F7CF911F914F
:101270000F91089566E085E00E9471070C944E0777
:10128000AF92BF92CF92DF92EF92FF920F931F9394
:1012900080911F01ECECF2E0219131912A3031056F
:1012A0000CF080E092E0EA3DF907B1F780931F016E
:1012B0006091DA027091DB02072E000C880B990B0B
:1012C0001F921F921F9221E12F93A12CB12C650137
:1012D000A394EE24EA9413E0F12E00E010E020E065
:1012E00030E0A9010E94261560931E010F900F9017
:1012F0000F900F901F910F91FF90EF90DF90CF9084
:10130000BF90AF900895CF92DF92EF92FF920F932C
:10131000CF93DF9300D0CDB7DEB77C016B010150D6
:10132000003108F05EC0603871050CF45AC0613EAF
:1013300071056CF5F70184A195A1DC01ED91FC919B
:10134000602B0190F081E02D2A8349830995F701F4
:1013500084A195A1DC01ED91FC914981642F6F7707
:101360000190F081E02D0995E894C4F82A81B0EC51
:10137000CB16D104B1F1F70184A195A1DC01ED9167
:10138000FC91622F6F770190F081E02D20C0CB019E
:10139000885F9109089728F56D3F71053CF46A3F15
:1013A00071054CF4683F7105E1F405C0CB018E5F17
:1013B00091090297B0F4D70194968D919C919597DD
:1013C000DC01ED91FC910190F081E02D6C2D0F90EE
:1013D0000F90DF91CF910F91FF90EF90DF90CF9022
:1013E00009940F900F90DF91CF910F91FF90EF90A4
:1013F000DF90CF9008950F93022F242F462F60EB9C
:1014000070E00E9483090F9108956F927F928F92EE
:101410009F92AF92BF92CF92DF92EF92FF920F9383
:101420001F93CF93DF933B01EC01CC0FDD1FCE0167
:1014300084539D4F4C01FC01608171818091240196
:10144000909125016817790709F48AC08091AD024F
:10145000813021F0873009F47BC04BC0072E000C8F
:10146000880B990B1F921F921F922FE72F93A12C8D
:10147000B12C6501EE24EA9413E0F12E00E010E0B7
:1014800020E030E0A9010E94261570931D016093B1
:101490001C01F401608171818091240190912501EA
:1014A0000E9434020F900F900F900F90882329F024
:1014B0008091BC02833008F419C120911C01309145
:1014C0001D01C90187559E4F880F991F880F991FCD
:1014D00090931B0180931A0189EA91E0821B930B80
:1014E000880F991F880F991F9093190180931801F5
:1014F0002FC0072E000C880B990B1F921F921F9272
:101500002FE72F93A12CB12C6501EE24EA9413E070
:10151000F12E00E010E020E030E0A9010E94261545
:101520007093AA026093A902F40160817181809195
:101530002401909125010E9434020F900F900F908A
:101540000F90882329F08091BC02833008F4D8C022
:10155000C453DD4F888199819093250180932401A4
:10156000E301CC0FDD1FCE0184539D4F4C01FC01E4
:101570006081718180912601909127016817790718
:1015800009F4DCC08091AD02813021F0873009F48C
:1015900046C075C0072E000C880B990B1F921F9236
:1015A0001F922DE02F93A12CB12C6501EE24EA941B
:1015B00013E0F12E00E010E020E030E0A9010E94ED
:1015C00026150F900F900F900F906D3071052CF431
:1015D0007093AC026093AB0206C08CE090E09093F5
:1015E000AC028093AB02FE01E453FD4F6081718138
:1015F00080912601909127010E943402882329F0CE
:101600008091BC02833008F485C02091160140917E
:10161000AB0264E18CED92E00E94FB095EC0809118
:10162000BC02823008F059C0072E000C880B990BC1
:101630001F921F921F9221E12F93A12CB12C6501C3
:10164000A394EE24EA9413E0F12E00E010E020E0F1
:1016500030E0A9010E9426150F900F900F900F9077
:10166000613118F46093160103C080E18093160184
:1016700081E00E94FE018091160190E05CC0072E7F
:10168000000C880B990B1F921F921F922FE72F932C
:10169000A12CB12C6501EE24EA9413E0F12E00E0B8
:1016A00010E020E030E0A9010E9426157093AC0202
:1016B0006093AB02F4016081718180912601909169
:1016C00027010E9434020F900F900F900F908823F3
:1016D00021F08091BC02833038F1C453DD4F888102
:1016E0009981909327018093260128C082E00E946F
:1016F000FE0180911C0190911D010E94E901DDCE47
:1017000082E00E94FE018091A9029091AA020E94AB
:10171000E9011ECF82E00E94FE018091AB02909110
:10172000AC020E94E90171CF82E00E94FE0180912B
:10173000AB029091AC020E94E901CFCFDF91CF9133
:101740001F910F91FF90EF90DF90CF90BF90AF90DF
:101750009F908F907F906F90089584E090E00E941A
:10176000550282E090E00E94D80265E070E086E0D9
:1017700090E00E94420381E090E00E948F0463E0C9
:1017800070E080E090E00C94050A64E070E082E094
:1017900090E00E94160563E070E080E090E00E9417
:1017A000050A65E070E086E090E00E94D50581E0E2
:1017B00090E00C948F044F925F926F927F92AF9261
:1017C000BF92CF92DF92EF92FF920F931F93CF932E
:1017D0006091B8027091B9028091BA029091BB02F7
:1017E0006115710581059105D1F1A090A902B09014
:1017F000AA020B2C000CCC08DD082091AB02309122
:10180000AC022901330F660877087F926F925F92CE
:101810004F9218EBE12E1BE0F12E00E010E02EE5D8
:1018200031E040E050E00E942615C62F0F900F9047
:101830000F900F9080910201C81789F08C2F90E0D3
:101840000E94E90181E00E94FE01209116014C2FC7
:1018500067E08CED92E00E94FB09C0930201CF91FA
:101860001F910F91FF90EF90DF90CF90BF90AF90BE
:101870007F906F905F904F9008954F925F926F921C
:101880007F92AF92BF92CF92DF92EF92FF920F932F
:101890001F93CF936091B8027091B9028091BA0200
:1018A0009091BB026115710581059105D1F1A09060
:1018B000A902B090AA020B2C000CCC08DD082091E4
:1018C000AB023091AC022901330F660877087F9292
:1018D0006F925F924F9218EBE12E1BE0F12E00E029
:1018E00010E02EE531E040E050E00E942615C62FC2
:1018F0000F900F900F900F9080911902C81789F0E8
:101900008C2F90E00E94E90181E00E94FE0120916D
:1019100016014C2F61E08CED92E00E94FB09C09310
:101920001902CF911F910F91FF90EF90DF90CF9010
:10193000BF90AF907F906F905F904F9008954F92BF
:101940005F926F927F92AF92BF92CF92DF92EF92AF
:10195000FF920F931F936091B8027091B90280912A
:10196000BA029091BB02611571058105910509F4D8
:1019700062C0A090A902B090AA020B2C000CCC0867
:10198000DD082091AB023091AC022901330F6608CB
:1019900077087F926F925F924F9218EBE12E1BE0D7
:1019A000F12E00E010E02EE531E040E050E00E9432
:1019B00026156093A2020F900F900F900F908091C8
:1019C00018026817C1F1862F90E00E94E90181E0BA
:1019D0000E94FE01209116014091A20265E08CED6B
:1019E00092E00E94FB098091A20281110DC020911A
:1019F000160140E061E48CED92E00E94FB098091C9
:101A0000A30281111092A3028091A30281110FC041
:101A10008091A202882359F0209116014FE761E4DA
:101A20008CED92E00E94FB0981E08093A3028091FB
:101A3000A202809318021F910F91FF90EF90DF9008
:101A4000CF90BF90AF907F906F905F904F90089530
:101A50004F925F926F927F92AF92BF92CF92DF923E
:101A6000EF92FF920F931F93CF936091B802709102
:101A7000B9028091BA029091BB026115710581058E
:101A8000910509F43FC0A090A902B090AA020B2CC6
:101A9000000CCC08DD082091AB023091AC0229018A
:101AA000330F660877087F926F925F924F9218EB20
:101AB000E12E1BE0F12E00E010E02EE531E040E0E9
:101AC00050E00E942615C62F0F900F900F900F9098
:101AD00080910101C81759F08091BC02811107C0A3
:101AE0008C2F90E00E94E90180E00E94FE0120918D
:101AF00016014C2F609122018CED92E00E94FB09AF
:101B0000C0930101CF911F910F91FF90EF90DF9053
:101B1000CF90BF90AF907F906F905F904F9008955F
:101B20004F925F926F927F92AF92BF92CF92DF926D
:101B3000EF92FF920F931F93CF938091BC0283305B
:101B400008F07DC06091B4027091B5028091B60238
:101B50009091B702611571058105910509F46FC077
:101B6000A090A502B090A6020B2C000CCC08DD08BA
:101B70002091A7023091A8022901330F6608770847
:101B80007F926F925F924F9218EBE12E1BE0F12E45
:101B900000E010E02EE531E040E050E00E94261524
:101BA000C62F0F900F900F900F9080910001C817D3
:101BB00059F08091BC02811107C08C2F90E00E94E7
:101BC000E90180E00E94FE01209116014C2F6091F6
:101BD00020018CED92E00E94FB09C09300018091EE
:101BE000B8029091B902A091BA02B091BB02892BC0
:101BF0008A2B8B2B21F18091B4029091B502A09198
:101C0000B602B091B702892B8A2B8B2BC1F088ECDE
:101C100090E0909331018093300180E38093CB0278
:101C20008FE28093CA0281E38093C90281E00E941F
:101C3000FE0180E293E09093310180933001CF91D7
:101C40001F910F91FF90EF90DF90CF90BF90AF90DA
:101C50007F906F905F904F9008950F9326E042E140
:101C60005AE760E070E080EA93E00E94071461E0C8
:101C700087E00E94591260E088E00E94591261E0FA
:101C800085E00E94591260E086E00E94591261E0EE
:101C900084E00E94591261E083E00E94591261E0E1
:101CA00082E00E94591260E083E10E94591261E0D3
:101CB0008EE00E94591261E08FE00E94591261E0AB
:101CC00089E00E94591261E082E10E94591261E0AC
:101CD00081E10E94591261E080E10E94591260EF97
:101CE00070E080910003909101030E94D7008091E1
:101CF000000390910103DC01ED91FC910190F081D2
:101D0000E02D60E009958091000390910103DC01D2
:101D1000ED91FC910190F081E02D60E0099567EF75
:101D200070E080910003909101030E94D700009120
:101D3000160120E041E560EC70E08CED92E00E943D
:101D400083090E94DE000E94400980911F018823C0
:101D500071F08DE28093CB028EE28093CA0282E022
:101D60008093C90288EE93E00E949A0102C00E940B
:101D7000160982E00F910C94FE01AF92BF92CF92B0
:101D8000DF92EF92FF920F931F93CF93DF93809197
:101D9000A2028823A1F01092A3021092A202209125
:101DA000160140E065E08CED92E00E94FB09209175
:101DB000160140E061E48CED92E00E94FB09609125
:101DC000B8027091B9028091BA029091BB02209141
:101DD0001A0130911B01032E000C440B550B2617E2
:101DE00037074807590788F4EFEFEF93EF93ECEFCD
:101DF000EF93E1E0EF93A12CB12C650118EBE12EFC
:101E00001BE0F12E00E010E01BC0E0901801F09004
:101E100019010F2C000C000B110B6E157F058007AC
:101E20009107B0F41F921F921F921F92AA24AA94A6
:101E300043E0B42EC12CD12C2EE531E040E050E03F
:101E40000E942615EB010F900F900F900F9002C08B
:101E5000C0E0D0E08091B8029091B902A091BA029E
:101E6000B091BB02892B8A2B8B2B11F580911C0220
:101E7000803118F48F5F80931C0280911C028F3098
:101E800009F0A9C08DE18093C90286E18093CA025E
:101E90008093CB0281E00E94FE010091160120E4B4
:101EA00040E060EE70E08CED92E00E94830993C008
:101EB00080911A0290911B02C817D90709F48BC0B0
:101EC0001C161D0644F5BE01C11584E0D80714F0A8
:101ED0006FEF73E0072E000C880B990B1F921F9277
:101EE0001F922DE12F9332E2A32EB12CC12CD12CC5
:101EF000E12CF12C87012FEF33E040E050E00E940D
:101F000026150F900F900F900F90CF3F83E0D807CA
:101F100099F56F5F31C0209791F1C1308CEFD807F0
:101F20005CF0BE011C161D0614F460E070E0072E84
:101F3000000C880B990B04C061E07CEF8FEF9FEFE2
:101F40001F921F921F922DE12F9328E1A22EB12CF8
:101F5000C12CD12CE12CF12C870121E03CEF4FEF7B
:101F60005FEF0E9426150F900F900F900F90C130D9
:101F70008CEFD80709F461506093030103C08DE131
:101F800080930301809103018093C90286E18093CD
:101F9000CA028093CB0281E00E94FE01D0931B0213
:101FA000C0931A0283E0CC0FDD1F8A95E1F7AE01E2
:101FB000505E9A01220F232F221F330B31952F776A
:101FC0004F770091160160EE70E08CED92E00E9478
:101FD000830910921C02DF91CF911F910F91FF9006
:101FE000EF90DF90CF90BF90AF9008958091BC02AA
:101FF0008230E0F48091AD02833081F028F48130AA
:1020000049F0823049F00895853061F048F086301B
:1020100059F008950C94BD0E0C943D0C0C941008CE
:102020000C94DB0B0C949F0C0C94280D0895CF930B
:10203000C0911E01CC2351F10E94E6068AE090E097
:102040000E949A010E943A090E9492076093B80286
:102050007093B9028093BA029093BB020E94F60F6C
:102060008091A402882381F00E940E090E94D1076A
:102070006093B4027093B5028093B6029093B70256
:102080000E94900D0E94C50BC150D4CFCF910895EE
:102090004F925F926F927F92AF92BF92CF92DF92F8
:1020A000EF92FF920F931F932B013C01672B682B3C
:1020B000692B39F586EF9FEF9093AF028093AE02C4
:1020C00080911702863018F48F5F809317028091F9
:1020D0001702863008F493C080911602882309F411
:1020E0008EC00091160120E04091150260E970E079
:1020F0008CED92E00E948309109217021092160252
:102100007EC0109217020E94C1116093C5027093A5
:10211000C6028093C7029093C802DC01CB01805AAB
:102120009541AF4FBF4F8093BD029093BE02A093E5
:10213000BF02B093C00280912F0190E00196092E5A
:10214000000CAA0BBB0BBF93AF939F938F93A12C53
:10215000B12C650118EBE12E1BE0F12E00E010E040
:102160002EE531E040E050E0C301B2010E942615A7
:1021700080912F010F900F900F900F90861708F409
:10218000682F70E07093AF026093AE02FB01EB5CCE
:10219000FD4F8081809314029091160291110FC01F
:1021A00091E0909316020091160120911701482F9B
:1021B00060E970E08CED92E00E9483091CC04091C0
:1021C00015028417E1F00091160120E060E970E04B
:1021D0008CED92E00E948309009116012091170175
:1021E0004091140260E970E08CED92E00E94830956
:1021F00081E08093160280911402809315021F9152
:102200000F91FF90EF90DF90CF90BF90AF907F90B5
:102210006F905F904F9008950E94DE000E94AC0680
:102220008091A402811106C00E94AD0B0E940E098C
:102230000C94481008950E940C110C941710CF9321
:10224000DF93ECEDF2E080EA93E095A384A316A27D
:1022500017A210A615A614A617A616A68FEF9FEF15
:1022600091AB80AB93AB82AB83E08093100315AA54
:1022700017AA16AA10AE11AE1092960380E8A6E136
:10228000B3E0ED0119928A95E9F711821082138269
:102290001282158214821782168211861086138686
:1022A00012861586148617861686118A108A138A56
:1022B000128A158A148A178A168A118E108E138E26
:1022C000128E158E148E178E168E11A210A213A2C6
:1022D00012A260912F0170E080ED92E00E948715BC
:1022E0007093B1026093B002DF91CF9108951F9275
:1022F0000F920FB60F9211242F933F938F939F93BA
:10230000AF93BF938091980390919903A0919A0302
:10231000B0919B033091970323E0230F2D3720F4D6
:102320000196A11DB11D05C026E8230F0296A11D2F
:10233000B11D209397038093980390939903A093E2
:102340009A03B0939B0380919C0390919D03A0916D
:102350009E03B0919F030196A11DB11D80939C0324
:1023600090939D03A0939E03B0939F03BF91AF9161
:102370009F918F913F912F910F900FBE0F901F90C3
:1023800018952FB7F89460919803709199038091F4
:102390009A0390919B032FBF08958230910538F0E6
:1023A000880F991F880F991F05970197F1F70895D6
:1023B000789484B5826084BD84B5816084BD85B520
:1023C000826085BD85B5816085BDEEE6F0E08081E7
:1023D00081608083E1E8F0E0108280818260808308
:1023E000808181608083E0E8F0E08081816080838B
:1023F000E1EBF0E0808184608083E0EBF0E08081BD
:1024000081608083EAE7F0E080818460808380815E
:102410008260808380818160808380818068808306
:102420001092C10008958E3008F08E508770209170
:10243000320190E4299F90011124822B80937C002B
:1024400080917A00806480937A0080917A0086FD82
:10245000FCCF809178002091790090E0922B089534
:10246000833081F028F4813099F08230A1F0089512
:102470008730A9F08830B9F08430D1F480918000A1
:102480008F7D03C0809180008F77809380000895B6
:1024900084B58F7702C084B58F7D84BD0895809107
:1024A000B0008F7703C08091B0008F7D8093B00023
:1024B0000895CF93DF9390E0FC01E158FF4F249102
:1024C000FC01EA56FF4F8491882361F190E0880F68
:1024D000991FFC01EF53FF4FC591D491FC01E954C2
:1024E000FF4FA591B491611109C09FB7F8948881FD
:1024F000209582238883EC912E230BC0623061F4F7
:102500009FB7F8943881822F809583238883EC913C
:102510002E2B2C939FBF06C08FB7F894E8812E2BEB
:1025200028838FBFDF91CF9108951F93CF93DF93BF
:10253000282F30E0F901E859FF4F8491F901E15863
:10254000FF4FD491F901EA56FF4FC491CC23C9F053
:10255000162F81110E943012EC2FF0E0EE0FFF1FBA
:10256000E954FF4FA591B4918FB7F894111105C0AC
:102570009C91ED2FE095E92302C0EC91ED2BEC93BB
:102580008FBFDF91CF911F9108950F931F9390E01C
:10259000FC01E158FF4F7491FC01EA56FF4FE491B2
:1025A000662311F0672F01C060E0F0E0EE0FFF1F1F
:1025B000E355FF4F8591949189019A013F70462F11
:1025C000672F0E949200611571058105910549F000
:1025D000DC01CB010196A11DB11DBC01CD019F7095
:1025E00003C060E070E0CB011F910F910895BF928E
:1025F000CF92DF92EF92FF920F931F93CF93DF93CF
:10260000C82ED62EB42EC7E0D0E0022F10E087E00F
:10261000E82EF12CB11005C0C7018C1B9D0B980151
:1026200002C098018C2F02C0359527958A95E2F754
:10263000B901617077278C2D0E94951261E08D2D74
:102640000E94951260E08D2D0E949512219710F73F
:10265000DF91CF911F910F91FF90EF90DF90CF907E
:10266000BF900895FC01918D228D892F90E0805CB0
:102670009F4F821B91098F7399270895FC01918DBB
:10268000828D981731F0828DE80FF11D858D90E0D5
:1026900008958FEF9FEF0895FC01918D828D98171B
:1026A00061F0828DDF01A80FB11D5D968C91928D36
:1026B0009F5F9F73928F90E008958FEF9FEF089533
:1026C000FC01538D448D252F30E0842F90E0821B38
:1026D000930B541710F0CF9608950197089584EC4A
:1026E00094E1892B49F080E090E0892B29F00E9449
:1026F000C41481110C9400000895FC01848DDF0145
:10270000A80FB11DA35ABF4F2C91848D90E0019664
:102710008F739927848FA689B7892C93A089B18953
:102720008C9180648C93938D848D981306C002885D
:10273000F389E02D80818F7D80830895CF93DF938F
:10274000EC01888D8823C9F0EA89FB89808185FDA9
:1027500005C0A889B9898C9186FD0FC00FB607FC0A
:10276000F5CF808185FFF2CFA889B9898C9185FF4B
:10277000EDCFCE010E947D13E7CFDF91CF91089579
:10278000EF92FF920F931F93CF93DF93EC0181E0C1
:10279000888F9B8D8C8D981305C0E889F98980817D
:1027A00085FD24C0F62E0B8D10E00F5F1F4F0F73B9
:1027B0001127E02E8C8DE8120CC00FB607FCFACF63
:1027C000E889F989808185FFF5CFCE010E947D13CC
:1027D000F1CF8B8DFE01E80FF11DE35AFF4FF08220
:1027E0000B8FEA89FB898081806207C0EE89FF89AF
:1027F0006083E889F98980818064808381E090E04A
:10280000DF91CF911F910F91FF90EF900895CF929C
:10281000DF92EF92FF921F93CF93DF93EC016A0157
:102820007B01122FE889F98982E080834115514E9E
:1028300061057105B1F060E079E08DE390E0A701FA
:1028400096010E949B15DA01C9010197A109B109FE
:10285000B695A79597958795AC01411580E15807E6
:10286000A8F0E889F989108260E874E88EE190E0C8
:10287000A70196010E949B15BA01A9014150510977
:10288000610971097695679557954795EC85FD85A2
:102890005083EE85FF854083188EEC89FD89108377
:1028A000EA89FB89808180618083EA89FB89808154
:1028B00088608083EA89FB89808180688083EA89D7
:1028C000FB8980818F7D8083DF91CF911F91FF9065
:1028D000EF90DF90CF9008951F920F920FB60F9256
:1028E00011242F938F939F93EF93FF93E091B00365
:1028F000F091B1038081E091B603F091B70382FDBE
:1029000012C090818091B9038F5F8F732091BA03B9
:10291000821751F0E091B903F0E0E056FC4F958F3B
:102920008093B90301C08081FF91EF919F918F91B6
:102930002F910F900FBE0F901F9018951F920F921E
:102940000FB60F9211242F933F934F935F936F9382
:102950007F938F939F93AF93BF93EF93FF9380EAFF
:1029600093E00E947D13FF91EF91BF91AF919F91F2
:102970008F917F916F915F914F913F912F910F9028
:102980000FBE0F901F90189580EA93E00E943213BB
:1029900021E0892B09F420E0822F0895E0EAF3E09A
:1029A0001382128288EE93E0A0E0B0E084839583E6
:1029B000A683B78385E092E09183808385EC90E0E5
:1029C0009587848784EC90E09787868780EC90E0F9
:1029D000918B808B81EC90E0938B828B82EC90E0EA
:1029E000958B848B86EC90E0978B868B118E128E64
:1029F000138E148E0895CF92DF92EF92FF920F9371
:102A00001F93CF93DF936C017A018B01C0E0D0E07C
:102A1000CE15DF0589F0D8016D918D01D601ED91BC
:102A2000FC910190F081E02DC6010995892B11F4EC
:102A30007E0102C02196ECCFC701DF91CF911F919B
:102A40000F91FF90EF90DF90CF9008954F925F929B
:102A50006F927F92AF92BF92CF92DF92EF92FF92EE
:102A60000F931F93CF93DF93CDB7DEB729013A01C0
:102A70009B01AC01241935094609570989899A89AE
:102A8000AB89BC89BC01CD016A197B098C099D0900
:102A90000E947715A801970124193509460957099D
:102AA0000E94BD15CA01B9016A0D7B1D8C1D9D1DBB
:102AB000DF91CF911F910F91FF90EF90DF90CF901A
:102AC000BF90AF907F906F905F904F900895089562
:102AD0000E94D8110E9467150E942D0ECFE6D3E107
:102AE0000E941B112097E1F30E946F13F9CFDB01C5
:102AF0008F939F930E94DC15BF91AF91A29F800D91
:102B0000911DA39F900DB29F900D1124089597FBE6
:102B1000072E16F4009407D077FD09D00E94E71520
:102B200007FC05D03EF4909581959F4F08957095D0
:102B300061957F4F0895A1E21A2EAA1BBB1BFD01D0
:102B40000DC0AA1FBB1FEE1FFF1FA217B307E4078C
:102B5000F50720F0A21BB30BE40BF50B661F771FE4
:102B6000881F991F1A9469F76095709580959095C4
:102B70009B01AC01BD01CF010895052E97FB1EF40A
:102B800000940E94D41557FD07D00E949B1507FCA6
:102B900003D04EF40C94D415509540953095219562
:102BA0003F4F4F4F5F4F0895909580957095619579
:102BB0007F4F8F4F9F4F08950E940116A59F900D44
:102BC000B49F900DA49F800D911D11240895AA1B00
:102BD000BB1B51E107C0AA1FBB1FA617B70710F008
:102BE000A61BB70B881F991F5A95A9F7809590953A
:102BF000BC01CD010895EE0FFF1F0590F491E02D6B
:102C00000994A29FB001B39FC001A39F700D811DC5
:102C10001124911DB29F700D811D1124911D0895E5
:042C2000F894FFCF56
:102C2400FFFF7F1DFFFFFFFFF5FF01000100FFFF16
:102C3400FFFFFFFFFFFF017FA406A4060A000101B6
:102C440056005500FFFFFFFF010200040005000FBE
:102C5400D007010202010202020100000000000785
:102C64000201020202010200000000000701020248
:102C74000201020200000000000702020201020237
:102C8400010000000000070202010202010200002C
:102C9400000000070201020201020200000000001D
:102CA4000701020201020202000000000007020103
:102CB40002020103010000000000070202030203F4
:102CC40000000000000000050302020302000000EF
:102CD40000000000050202020202020000000000DF
:102CE40000060101010101010101010101010CAF13
:102CF400289BBA3CB6B72ABFBE87C7B9F9971757FE
:102D0400B7F73F7FB500EFAFAEAAA8A08081858753
:102D14008FAFEFFEFDFBF7EFDFBF7FFFDB68101522
:102D24003800000000C013FB1460139E1332134CD0
:042D3400133E130037
:00000001FF
